:100000007B2964001720031801285620A801083016
:10001000A300572017200318A80AAB1EA801A20CA2
:10002000A30B0928AB1AA2135720220808003A088C
:100030008400380884178004841300052B1B3806BD
:10004000FF3E08000408A6003A088400F030B70517
:100050000830A70003100318B70A3C20A60CA70B12
:100060002B280000AB1A370C3C20792103143C20CC
:100070002F08A3002E08D7288413AB1F4B28000895
:1000800038042B1F38068000841700083804031C2E
:1000900038068000572800083804031C38062B1B3C
:1000A00038068000841738098005572837172B0831
:1000B0001F39FF3EA1002A08F53E0318A10A371F89
:1000C000E4283713A00002301621E428B7132908CA
:1000D0000319B7170530A8002730A30010307C2083
:1000E0000330A300E8307C20A30164307C20A3010E
:1000F0000A307C2024088328A2002508A1002408B7
:10010000A0003F212008A000A8030319B713290865
:1001100003198D282802031808002008031DB713AF
:10012000B71B0800303E71290830A6003718F820A8
:100130003B08840039083719B720371DB9203A0821
:1001400084003809BD203A088400A10CA00C0008E6
:100150003804031C38068000B020A60BA32876299B
:100160003B088400390880060000800608008004EF
:10017000BC28FF3A8005BD28FF3A84178005762900
:1001800003178D0083168C130C1483120C08762928
:1001900003178C0083168C130C1555308D00AA3074
:1001A0008D008C148C18D2280C117629A301A20082
:1001B000FF30A207031CA307031C76290330A1000C
:1001C000DF30E420D828A101E83EA000A109FC30DE
:1001D000031CED28A0070318EA28A0076400A10F5C
:1001E000EA282018F328A01CF7280000F7280800A8
:1001F000A400A201A3010029A10CA00CA20DA30D33
:10020000FF3E0318FC2824080E212208A00423081E
:10021000A104200808000310A00DA10DFF3E031843
:100220000B29200876290310A10CA00CFF3E03180F
:10023000132920087629A101A301A2000130282951
:10024000A20006302829A101A301A2000430282918
:10025000A80023082102031D2F29220820020430B0
:1002600003180130031902302805031DFF307629D9
:100270000038031DFF300405031DFF3076291030C0
:10028000A600A501A401210DA40DA50D2208A4021C
:100290002308031C230FA502031855292208A407CD
:1002A00023080318230FA5070310A00DA10DA60B0B
:1002B0004329200876291030A800A101A001A70C2D
:1002C000A60C031C69292208A00723080318230F82
:1002D000A107A10CA00CA50CA40CA80B5F29240855
:1002E0007629840031088A003008820083130313C2
:1002F000831264000800831601308600850187019F
:100300008312E330DE00DA010230DB000730BA008E
:100310000230B8005430AA004030AB00AE01AF014B
:1003200050308A01232072308A01232075308A01DF
:10033000232065308A01232062308A012320613026
:100340008A01232073308A01232020308A01232050
:1003500073308A01232069308A0123206E308A019C
:10036000232074308A01232065308A0123207430D1
:100370008A01232069308A0123207A308A012320D0
:1003800061308A01232064308A0123206F308A0182
:10039000232072308A01232020308A01232050300C
:1003A0008A01232049308A01232043308A012320F7
:1003B0002D308A01232054308A01232072308A0193
:1003C000232061308A0123206E308A01232073307C
:1003D0008A01232063308A01232065308A0123208B
:1003E00069308A01232076308A01232065308A0112
:1003F000232072308A01232020308A0123202D30CF
:100400008A01232020308A01232045308A012320BD
:1004100041308A01232033308A01232043308A016E
:1004200023204E308A0123204F308A0123200A30B6
:100430008A0123200D308A01232000308A01C02048
:10044000E00001308A01C020E1006008A600A70199
:100450006430A200A3018A015B21B2002508B30029
:1004600061083207DC0033080318013EDD008A1101
:100470000A1261250A308A01D6200730BA000230FC
:10048000B8005430AA004030AB00AE01AF0141309B
:100490008A0123206A308A01232075308A012320B3
:1004A00073308A01232074308A01232065308A0149
:1004B000232020308A01232066308A0123207230D5
:1004C0008A01232065308A01232063308A0123209A
:1004D00075308A01232065308A0123206E308A011D
:1004E000232063308A01232069308A012320613070
:1004F0008A01232020308A01232068308A012320AA
:100500003D308A01232035308A01232030308A0192
:10051000232030308A01232020308A0123204B30D1
:100520008A01232048308A0123207A308A0123203F
:1005300020308A0123206C308A0123203D308A013B
:10054000232032308A01232035308A0123204B308A
:100550008A01232048308A0123207A308A0123200F
:1005600020308A01232066308A0123203D308A0111
:10057000232031308A01232034308A012320343073
:100580008A0123202E308A01232030308A01232043
:1005900030308A01232030308A0123204D308A01F7
:1005A000232048308A0123207A308A0123200A3010
:1005B0008A0123200D308A0123200730BA00013040
:1005C000B8005430AA004030AB008A010120E2009C
:1005D0006208A00069308A012321B2006208A000ED
:1005E00067308A011B21B4003208840034088A0174
:1005F00038218A110A12031D292B6208A0006D30D0
:100600008A012321B2006208A0006B308A011B21FD
:10061000B4003208840034088A0138218A110A1291
:10062000031DD52B6208A00067308A012321B20088
:100630006208A00065308A011B21B40032088400E2
:1006400034088A0138218A110A12031DA22D8A0159
:100650003D2A0730BA000230B8005430AA004030BA
:10066000AB00AE01AF012B308A0123202F308A016D
:1006700023202D308A01232020308A012320353089
:100680008A01232030308A01232030308A01232040
:1006900020308A0123204B308A01232048308A01F0
:1006A00023207A308A01232020308A012320203021
:1006B0008A0123206D308A0123203D308A012320C6
:1006C0004D308A01232065308A0123206E308A0153
:1006D000232075308A0123200A308A0123200D301F
:1006E0008A0123200730BA000130B8005430AA0034
:1006F0004030AB008A010120E300FA308A01D620A5
:100700006308A0002C308A012321B2006308A000F6
:100710002A308A011B21B4003208840034088A017F
:1007200038218A110A12031DC12B6308A0002E3044
:100730008A012321B2006308A0002C308A011B210A
:10074000B4003208840034088A0138218A110A1260
:10075000031DCA2B6308A0006E308A012321B2005A
:100760006308A0006C308A011B21B40032088400A9
:1007700034088A0138218A110A12031D3D2A8A0190
:10078000292B2830DC070318DD0A8A110A1261259B
:100790008A01292B2830DC020030031C013EDD02D7
:1007A0008A110A1261258A01292B0730BA0002300A
:1007B000B8005430AA004030AB00AE01AF012B307E
:1007C0008A0123202F308A0123202D308A01232003
:1007D00020308A01232032308A01232035308A01DB
:1007E000232020308A0123204B308A0123204830E7
:1007F0008A0123207A308A01232020308A01232095
:1008000020308A0123206D308A0123203D308A0167
:1008100023204D308A01232065308A0123206E3049
:100820008A01232075308A0123200A308A0123207F
:100830000D308A0123200730BA000130B80054304F
:10084000AA004030AB008A010120E300FA308A019F
:10085000D6206308A0002C308A012321B20063084F
:10086000A0002A308A011B21B40032088400340819
:100870008A0138218A110A12031D6A2C6308A0001C
:100880002E308A012321B2006308A0002C308A0197
:100890001B21B4003208840034088A0138218A11EF
:1008A0000A12031D732C6308A0006E308A012321F5
:1008B000B2006308A0006C308A011B21B40032082A
:1008C000840034088A0138218A110A12031D3D2A46
:1008D0008A01D52B0230DC070318DD0A8A110A12BF
:1008E00061258A01D52B0230DC020030031C013E59
:1008F000DD028A110A1261258A01D52B8612831620
:10090000861206308312BA004030B8000630BB00B1
:100910001030B9000130B7005E08A000A1018A01C3
:1009200094208616831686120A3083128A01D620F6
:1009300086128316861206308312BA004030B80041
:100940000630BB001030B9000130B7005A08A000D3
:100950005B08A1000F308A01952086168316861247
:100960000A3083128A01D6208612831686128312D9
:100970000616831606128312061283160612063016
:100980008312BA004030B8000630BB001030B90006
:100990000130B7005C08A0005D08A1000F308A019B
:1009A000952086168316861283125C08A0005D08C7
:1009B000A1006430A200A3018A013F21E0005C088D
:1009C000A0005D08A1006430A200A3018A013F21BC
:1009D0002408E10003178D01031360088A01C82071
:1009E000031701308D00031361088A01C8203230DB
:1009F0008A01D6200800A0305C02B2002830031C17
:100A0000013E5D02B3003208A6003308A70019308A
:100A1000A200A3018A015B21B2002508B3000310E4
:100A2000330CBD00320CBC00A0305C02B200283098
:100A3000031C013E5D02B3003208A6003308A70084
:100A40001930A200A3018A015B21B2002508B3007E
:100A50003208A0003308A1000230A200A3018A01DD
:100A60003F212408B2002508B3003208A60033084D
:100A7000A7000530A200A3018A015B21BE00250862
:100A8000BF005C08A0005D08A1002B30A300BF30B0
:100A90008A011D218A110A12031D5B2D5C08A0002A
:100AA0005D08A1002B30A300BF308A0120218A11EC
:100AB0000A12031D5E2D0E30DF0008000D30DF002E
:100AC00008008A017E248A01FB240730BA00023024
:100AD000B8005430AA004030AB00AE01AF01023084
:100AE000A9005F08A400A5012230B000B1018A016D
:100AF00066200430A9003C08A4003D08A50022306F
:100B0000B000B1018A0166202E308A012320013015
:100B1000A9003E08A4003F08A5002230B000B101A2
:100B20008A0166204D308A01232048308A01232023
:100B30007A308A0123200A308A0123200D308A016D
:100B400023200800DC012D30DD008A0161258A01A7
:080B50003D2A63008A01A92D72
:02400E00753DFE
:00000001FF
